:100000000EC028C027C026C025C024C023C022C0DF
:1000100021C020C01FC01EC01DC01CC01BC0112499
:100020001FBECFE5D2E0DEBFCDBF10E0A0E6B0E05E
:10003000E8E5FDE102C005900D92A438B107D9F7BB
:1000400011E0A4E8B0E001C01D92A231B107E1F7D0
:10005000F9D981CED5CF89E288BB08952091790066
:1000600030917A0040917B0050917C00F7DD20E0D8
:1000700030E040E050E004C02F5F3F4F4F4F5F4FF4
:100080006217730784079507BCF72093D800309355
:10009000D9004093DA005093DB00089589E288BBD1
:1000A00061E070E080E090E0D9DF88E288BB0895ED
:1000B00020917D0030917E0040917F005091800022
:1000C000CDDD20E030E040E050E004C02F5F3F4F46
:1000D0004F4F5F4F6217730784079507BCF7209354
:1000E000DC003093DD004093DE005093DF00089584
:1000F0001F9318BA81E087BB19E218BB68EE73E062
:1001000080E090E0ABDF83E087BB18BB61E070E08C
:1001100080E090E0A3DF1F91089583E087BB89E230
:1001200088BB0895662391F4853011F417B83EC05A
:10013000823011F481E039C0843011F482E035C09E
:10014000833099F18A3091F58DE02FC06130A1F4B0
:10015000853011F480E929C0823011F481E925C08D
:10016000843011F482E921C0833011F483E91DC089
:100170008A30E1F48DE919C06230C1F4853011F4A0
:1001800080E813C0823011F481E80FC0843011F48C
:1001900082E80BC0833011F483E807C08A3011F481
:1001A0008DE803C08B3011F48FE887B986EC86B9EF
:1001B0003699FECF84B195B19C0140E050E0209388
:1001C000AA003093AB004093AC005093AD0066237F
:1001D00019F58091B2009091B300A091B400B09154
:1001E000B500281B390B4A0B5B0B2093AA003093F8
:1001F000AB004093AC005093AD0057FF08C0109285
:10020000AA001092AB001092AC001092AD0020E258
:100210003EE440E050E05AC06130A1F58091B60064
:100220009091B700A091B800B091B900281B390B8C
:100230004A0B5B0B2093AA003093AB004093AC00B9
:100240005093AD0057FF08C01092AA001092AB0067
:100250001092AC001092AD002AE030E040E050E097
:100260006091AA007091AB008091AC009091AD00BC
:10027000F5DC6093AA007093AB008093AC00909380
:10028000AD003AC06230C1F58091BA009091BB00D8
:10029000A091BC00B091BD00281B390B4A0B5B0B31
:1002A0002093AA003093AB004093AC005093AD0074
:1002B00057FF08C01092AA001092AB001092AC0039
:1002C0001092AD002CE434E040E050E06091AA00D0
:1002D0007091AB008091AC009091AD00BFDC2FEF2E
:1002E00033E040E050E0E6DC2093AA003093AB001E
:1002F0004093AC005093AD006091AA007091AB00A8
:100300008091AC009091AD0008951092B2001092CF
:10031000B3001092B4001092B50060E08AE002DFF2
:1003200084B195B1A0E0B0E08093B2009093B300A7
:10033000A093B400B093B5001092B6001092B7002D
:100340001092B8001092B90061E08AE0EBDE84B14F
:1003500095B1A0E0B0E08093B6009093B700A09371
:10036000B800B093B9001092BA001092BB0010927E
:10037000BC001092BD0062E08AE0D4DE84B195B189
:10038000A0E0B0E08093BA009093BB00A093BC00C3
:10039000B093BD00089589E288BB61E070E080E021
:1003A00090E05CDE10929D0010929E0010929F00E3
:1003B0001092A00021C08BE288BB64E170E080E075
:1003C00090E076DE89E288BB69E170E080E090E051
:1003D00045DE80919D0090919E00A0919F00B0917C
:1003E000A0000196A11DB11D80939D0090939E00D9
:1003F000A0939F00B093A00060916D0070916E007B
:1004000080916F009091700022E330E040E050E076
:1004100051DC80919D0090919E00A0919F00B09131
:10042000A00082179307A407B5072CF20895E1995D
:10043000FECF1CBA90E09FBB8EBB6DBBE29AE19AE7
:100440000895E199FECF90E09FBB8EBBE09A8DB3FB
:1004500090E0089564EF71E080E090E0FFDD9BDFC5
:100460001092E9001092EA001092EB001092EC005A
:100470001092AE001092AF001092B0001092B10036
:1004800056C060E084E04EDE645F71408040904082
:1004900014F41092C60060E084E044DE2091640011
:1004A000309165004091660050916700261737072C
:1004B000480759074CF58091C600882329F580919B
:1004C000E9009091EA00A091EB00B091EC00019658
:1004D000A11DB11D8093E9009093EA00A093EB0069
:1004E000B093EC0080938200843018F083E0809316
:1004F00082001092AE001092AF001092B0001092E5
:10050000B10081E08093C6008091AE009091AF0071
:10051000A091B000B091B1000196A11DB11D8093D2
:10052000AE009093AF00A093B000B093B100809163
:10053000AE009091AF00A091B000B091B10088558D
:100540009240A040B0400CF49CCF25DF6AEF70E0F1
:1005500080E090E083DD1FDF1092AE001092AF00CC
:100560001092B0001092B10054C060E084E0DADD77
:10057000645F71408040904014F41092C60060E0C7
:1005800084E0D0DD209164003091650040916600E8
:100590005091670026173707480759073CF58091A7
:1005A000C600882319F58091680090916900A09198
:1005B0006A00B0916B00181619061A061B06B4F4EF
:1005C0000197A109B1098093680090936900A093F5
:1005D0006A00B0936B001092AE001092AF001092C0
:1005E000B0001092B10081E08093C6008091AE000F
:1005F0009091AF00A091B000B091B1000196A11D03
:10060000B11D8093AE009093AF00A093B000B09363
:10061000B1008091AE009091AF00A091B000B09178
:10062000B10088559240A040B0400CF49ECFB3DE9C
:100630006AEF70E080E090E011DDADDE6AEF70E01F
:1006400080E090E00BDDA7DE1092AE001092AF00CC
:100650001092B0001092B10054C060E084E062DDFE
:10066000645F71408040904014F41092C60060E0D6
:1006700084E058DD2091640030916500409166006F
:100680005091670026173707480759073CF58091B6
:10069000C600882319F58091680090916900A091A7
:1006A0006A00B0916B008A3F9105A105B105B4F4D1
:1006B0000196A11DB11D8093680090936900A093DD
:1006C0006A00B0936B001092AE001092AF001092CF
:1006D000B0001092B10081E08093C6008091AE001E
:1006E0009091AF00A091B000B091B1000196A11D12
:1006F000B11D8093AE009093AF00A093B000B09373
:10070000B1008091AE009091AF00A091B000B09187
:10071000B10088559240A040B0400CF49ECF3BDE23
:100720006AEF70E080E090E099DC35DE6AEF70E01F
:1007300080E090E093DC2FDE6AEF70E080E090E0F4
:100740008DDC29DE1092AE001092AF001092B00046
:100750001092B10051C060E084E0E4DC645F71405D
:100760008040904014F41092C60060E084E0DADC2F
:1007700020916400309165004091660050916700BF
:10078000261737074807590724F58091C6008823A4
:1007900001F580916C008823E1F090E069E070E061
:1007A0004BDA6AE070E073DA60936C001092AE008E
:1007B0001092AF001092B0001092B1001092E000C1
:1007C0001092E1001092E2001092E30081E0809329
:1007D000C6008091AE009091AF00A091B000B091A2
:1007E000B1000196A11DB11D8093AE009093AF00A2
:1007F000A093B000B093B1008091AE009091AF0093
:10080000A091B000B091B10088559240A040B04096
:100810000CF4A1CFC0DD6AEF70E080E090E01EDC58
:10082000BADD6AEF70E080E090E018DCB4DD6AEFDA
:1008300070E080E090E012DCAEDD6AEF70E080E016
:1008400090E00CDCA8DD1092AE001092AF00109288
:10085000B0001092B10057C060E084E063DC645FD8
:1008600071408040904014F41092C60060E084E033
:1008700059DC2091640030916500409166005091F0
:100880006700261737074807590754F58091C600B7
:10089000882331F580916C008F3F11F1883E50F430
:1008A00090E06BE070E0C8D96AE070E0F0D9609346
:1008B0006C0003C08EEF80936C001092AE0010921B
:1008C000AF001092B0001092B1001092E0001092B0
:1008D000E1001092E2001092E30081E08093C600F4
:1008E0008091AE009091AF00A091B000B091B100A6
:1008F0000196A11DB11D8093AE009093AF00A0930F
:10090000B000B093B1008091AE009091AF00A09183
:10091000B000B091B10088559240A040B0400CF4B6
:100920009BCF6091820081E082DD80916800909190
:100930006900A0916A00B0916B00C297A105B10552
:1009400064F482E390E0A0E0B0E0809368009093CC
:100950006900A0936A00B0936B0080916800909149
:100960006900A0916A00B0916B008B3F9105A105D1
:10097000B10564F08AEF90E0A0E0B0E080936800F9
:1009800090936900A0936A00B0936B006091680037
:1009900082E04DDD80916C00843318F484E3809311
:1009A0006C0080916C008F3F19F48EEF80936C0087
:1009B00060916C0084E03BDD609184007091850063
:1009C000809186009091870024E630E040E050E07E
:1009D00071D92093ED00622F85E029DDDCDC6AEF20
:1009E00070E080E090E03ADBD6DC6AEF70E080E017
:1009F00090E034DBD0DC6AEF70E080E090E02EDB4A
:100A0000CADC6AEF70E080E090E028DBC4DC6AEFCB
:100A100070E080E090E022DBBEDC1092E5001092F6
:100A2000E6001092E7001092E8001092AE001092DB
:100A3000AF001092B0001092B10059C08091E50053
:100A40009091E600A091E700B091E8000196A11D09
:100A5000B11D8093E5009093E600A093E700B0936A
:100A6000E8008D5D9540A040B040ECF06FEF80E075
:100A7000DEDC6FEF81E0DBDC6FEF82E0D8DC6FEF74
:100A800083E0D5DC6FEF84E0D2DC6FEF85E0CFDC74
:100A900082DC81DC80DC7FDC7EDC7DDC7CDC7BDC82
:100AA0007ADC79DCFFCF60E084E03CDB20916400FD
:100AB0003091650040916600509167002617370716
:100AC000480759070CF4BACF8091AE009091AF005F
:100AD000A091B000B091B1000196A11DB11D80930D
:100AE000AE009093AF00A093B000B093B10080919E
:100AF000AE009091AF00A091B000B091B1008855C8
:100B00009240A040B0407CF208956F927F928F9205
:100B10009F92AF92BF92CF92DF92EF92FF920F938C
:100B20001F9362E180E083DC81E08BDC8F3F21F06A
:100B300081E087DC8093820082E083DC8F3F69F074
:100B400082E07FDC90E0A0E0B0E0809368009093CA
:100B50006900A0936A00B0936B0083E072DC8F3F62
:100B600009F46BC083E06DDC682E77248824992417
:100B70006092710070927200809273009092740083
:100B80001092E0001092E1001092E2001092E30057
:100B9000E0906800F090690000916A0010916B008D
:100BA000EE0CFF1C001F111F84E690E0A0E0B0E0F7
:100BB000E80EF91E0A1F1B1FE0928800F0928900C0
:100BC00000938A0010938B0025E730E040E050E06E
:100BD000C801B70143D8A401930140D820EE3EE2FA
:100BE00040E050E067D859016A0125E230E040E07A
:100BF00050E0C801B70132D864577E408040904031
:100C000028E730E040E050E055D8A20EB31EC41EE5
:100C1000D51EA0927500B0927600C0927700D09257
:100C2000780080918200833041F460927500709268
:100C30007600809277009092780084E002DC8093C6
:100C40006C0085E0FEDB8F3F91F085E0FADB90E001
:100C500064E670E0F1D7AA2797FDA095BA2F80939C
:100C6000840090938500A0938600B09387001F9125
:100C70000F91FF90EF90DF90CF90BF90AF909F903B
:100C80008F907F906F9008956F927F928F929F9236
:100C9000AF92BF92CF92DF92EF92FF920F931F938A
:100CA0003B014C018091E0009091E100A091E200B5
:100CB000B091E3000196A11DB11D8093E0009093D7
:100CC000E100A093E200B093E30083309105A10519
:100CD000B10549F4609271007092720080927300C5
:100CE0009092740036C00497A105B10594F1E0908C
:100CF0007100F090720000917300109174002BE06D
:100D000030E040E050E0C801B701A8D72AE030E069
:100D100040E050E0CFD726153705480559050CF4BB
:100D20001BC1C801B701F3E0660F771F881F991F29
:100D3000FA95D1F76E0D7F1D801F911F2AE030E0DC
:100D400040E050E0B7D762167306840695063CF57E
:100D500003C1209171003091720040917300509155
:100D60007400CA01B901E2E0660F771F881F991F5E
:100D7000EA95D1F7620F731F841F951F660D771DCB
:100D8000881D991D26E030E040E050E093D7209385
:100D90007100309372004093730050937400E090A0
:100DA0006800F090690000916A0010916B00EE0CF1
:100DB000FF1C001F111F84E690E0A0E0B0E0E80EE9
:100DC000F91E0A1F1B1FE0928800F0928900009311
:100DD0008A0010938B006090710070907200809078
:100DE00073009090740025E230E040E050E0C801CC
:100DF000B70134D764577E408040904028E730E008
:100E000040E050E057D759016A0125E730E040E063
:100E100050E0C401B30122D7A80197011FD720EEEB
:100E20003EE240E050E046D72A0D3B1D4C1D5D1DC3
:100E300020937500309376004093770050937800AC
:100E4000261537054805590544F4609275007092DF
:100E50007600809277009092780097FE0CC081E037
:100E600090E0A0E0B0E08093710090937200A093B6
:100E70007300B09374008091710090917200A09102
:100E80007300B09174008F3F9105A105B10564F026
:100E90008EEF90E0A0E0B0E080937100909372003C
:100EA000A0937300B0937400209171003091720090
:100EB000409173005091740080918C0090918D004E
:100EC000A0918E00B0918F00281739074A075B0761
:100ED00099F0622F83E0ABDA8091710090917200FB
:100EE000A0917300B091740080938C0090938D005A
:100EF000A0938E00B0938F008091E0009091E1006C
:100F0000A091E200B091E3000397A105B1056CF454
:100F10008091710090917200A0917300B091740063
:100F2000880F991FAA1FBB1F0FC0809182008330BA
:100F300099F48091710090917200A0917300B0912A
:100F400074000297A109B10980937500909376000F
:100F5000A0937700B09378001F910F91FF90EF90CE
:100F6000DF90CF90BF90AF909F908F907F906F90C9
:100F70000895982F882339F483E08ABD80E88CBDDA
:100F800089E288BB089581E88CBD83E28ABD81E057
:100F900083BF92BF98BD88E089BF1CBC089580E0E4
:100FA000E8DF08951F93803150F4182F105C812FD3
:100FB00048DA8F5F8093FE00682F812F38DA1F9107
:100FC00008951F9360E084E0ADD86093F7007093BC
:100FD000F8008093F9009093FA00685271418040C4
:100FE0009040615D73408040904008F0CEC080E04A
:100FF000D9DF8BE287BB81E088BB11E01093FB0057
:1010000018BB60ED77E080E090E028D860E084E0F5
:1010100089D86093F7007093F8008093F90090935B
:10102000FA006E5772418040904064527140804097
:10103000904018F082E08093FB0061E084E072D879
:101040006093F7007093F8008093F9009093FA0092
:101050006E57724180409040645271408040904091
:1010600018F083E08093FB0061E082E05BD860933E
:10107000F7007093F8008093F9009093FA006E5790
:10108000724180409040645271408040904018F01E
:1010900084E08093FB0083E088BB61E070E080E047
:1010A00090E0DCD761E082E03DD86093F700709378
:1010B000F8008093F9009093FA006B307105810578
:1010C000910518F085E08093FB0018BB61E070E0AB
:1010D00080E090E0C3D718BA61E070E080E090E073
:1010E000BDD761E082E01ED86093F7007093F800EE
:1010F0008093F9009093FA00655E754280409040BD
:10110000695572408040904018F086E08093FB0063
:1011100018BB61E070E080E090E0A0D71092FC0086
:1011200013C081E288BB64EF71E080E090E096D765
:1011300081E088BB64EF71E080E090E08FD7809120
:10114000FC008F5F8093FC009091FB008091FC007D
:10115000891738F3913009F450CF6CED75E080E0D9
:1011600090E07CD781E288BB6091F7007091F80035
:101170008091F9009091FA0071D781E088BB60ED11
:1011800077E080E090E06AD738CF1F9108952F92E2
:101190003F924F925F926F927F928F929F92AF9207
:1011A000BF92CF92DF92EF92FF920F931F9319E2BB
:1011B00018BB61E070E080E090E050D78BE288BB24
:1011C00061E070E080E090E049D761E082E0AAD77A
:1011D0006093950070939600809397009093980089
:1011E00018BB28EE33E040E050E038D5625F7D4F19
:1011F0008A4090403CF018BB82E0D4DE81E18093CD
:1012000090004CC081E0B5DE90916C00892F8695EE
:10121000282E3324442455242091F3003091F400E7
:101220004091F5005091F600692E77248824992486
:10123000EE24FF248701AA24BB24650115C0C60142
:10124000B501661977098809990924E630E040E07C
:1012500050E030D5220D331D441D551D28BD089486
:10126000E11CF11C011D111DA60CB71CC81CD91CCA
:1012700083E3E816F104010511050CF32093F30054
:101280003093F4004093F5005093F600E092EF00A5
:10129000F092F0000093F1001093F2001F910F9173
:1012A000FF90EF90DF90CF90BF90AF909F908F9086
:1012B0007F906F905F904F903F902F90089589E2BC
:1012C00088BB61E070E080E090E0C8D660E083E039
:1012D00029D724E030E040E050E0ECD42093000136
:1012E00030930101409302015093030160E085E0D7
:1012F00019D724E030E040E050E0DCD42093040132
:10130000309305014093060150930701809100013D
:1013100090910101A0910201B09103018C3261E032
:10132000960760E0A60760E0B60774F42C3261E02F
:10133000360760E0460760E0560734F481E08093AA
:10134000080181E090E00895255F31404040504021
:101350001CF083E090E00895855F9140A040B0408C
:101360001CF082E090E0089581E090E00895EF9213
:10137000FF920F931F937B018C01FFE0EE0CFF1C8B
:10138000001F111FFA95D1F72FEF3FEF4FEF5FE7E7
:10139000E222F322042315239B01AC01E5E15595DC
:1013A000479537952795EA95D1F7E21AF30A040B8A
:1013B000150B9C01552737FD5095452FE20EF31E66
:1013C000041F151FAAE0660F771F881F991FAA9593
:1013D000D1F79F77E61AF70A080B190B17FF08C019
:1013E0008FEF9FEFAFEFBFE7E80EF91E0A1F1B1F3D
:1013F000C801B7011F910F91FF90EF90089589E206
:1014000088BB61E070E080E090E028D660E083E097
:1014100089D624E030E040E050E04CD42093000135
:1014200030930101409302015093030190E0295B46
:101430003B40404050400CF091E081E09827892FDC
:1014400090E00895DF92EF92FF920F931F9360ED6B
:1014500077E080E090E002D681E08093900002E0A7
:101460000093810052D760E084E05CD6655F7140F4
:10147000804090401CF084E08093900046DB38D69A
:1014800013E017BB89E288BB60E082E04BD6609333
:10149000990070939A0080939B0090939C0068350C
:1014A0002BE1720720E0820720E0920714F40093FA
:1014B0009000695672448040904024F081E072DDD3
:1014C000109390008091840090918500A0918600F7
:1014D000B09187000097A105B10559F460E082E062
:1014E00021D660938400709385008093860090934A
:1014F0008700E0908400F0908500009186001091B4
:10150000870020E530E040E050E0C801B701A6D3F5
:1015100024E630E040E050E0CDD3209364003093E7
:101520006500409366005093670025E530E040E099
:1015300050E0C801B70192D324E630E040E050E02B
:10154000B9D32093600030936100409362005093C0
:1015500063001092FF00109208011092D4001092C4
:10156000D5001092D6001092D70019C064EF71E038
:1015700080E090E073D50FD78091D4009091D50092
:10158000A091D600B091D7000196A11DB11D809306
:10159000D4009093D500A093D600B093D70080914B
:1015A000900090E0A0E0B0E02091D4003091D50010
:1015B0004091D6005091D700281739074A075B079A
:1015C000ACF2FFDC809190008230F0F71092AE0018
:1015D0001092AF001092B0001092B10024C060E0F1
:1015E00084E0A0D5209164003091650040916600B0
:1015F0005091670026173707480759070CF42AD778
:101600008091AE009091AF00A091B000B091B10078
:101610000196A11DB11D8093AE009093AF00A093E1
:10162000B000B093B1008091AE009091AF00A09156
:10163000B000B091B100815A9440A040B0407CF21B
:10164000AAD6A9D6A8D6A7D680910801882321F0CA
:10165000A2D6A1D6A0D69FD68091C7009091C800EF
:10166000A091C900B091CA000196A11DB11D80933F
:10167000C7009093C800A093C900B093CA0080919E
:101680000A0190910B01A0910C01B0910D010196FE
:10169000A11DB11D80930A0190930B01A0930C0131
:1016A000B0930D017CDC8091CF00813069F4A7DE1E
:1016B000882351F01092CF001092CB001092CC00F2
:1016C0001092CD001092CE0060E084E02BD59B01FB
:1016D000AC0160939100709392008093930090937B
:1016E00094008091640090916500A0916600B09193
:1016F000670082179307A407B507ECF58091C60031
:101700008823C9F5809108018823A9F4809160009D
:1017100090916100A0916200B09163002817390791
:101720004A075B076CF48091EE008F5F8093EE00B8
:101730008330E8F4A5C0C3DD8093FF00813019F445
:101740001092EE009DC09091EE009F5F9093EE008E
:10175000833039F4933008F493C080E18093900093
:10176000D5C1823009F08CC0933008F489C080E183
:101770008093900085C0245F3140404050406CF41D
:101780001092C60081E0809381001092C7001092F1
:10179000C8001092C9001092CA008091C7009091B1
:1017A000C800A091C900B091CA00883A9105A1056E
:1017B000B10564F08091C600813041F480918200CF
:1017C000833021F082E0809381005AC0809109012A
:1017D000882309F041CF8091BE009091BF00A09175
:1017E000C000B091C1008D529140A040B04008F4BB
:1017F00033CF80910A0190910B01A0910C01B0911F
:101800000D01895E9340A040B0400CF425CF60E00C
:1018100082E088D47B018C01609384007093850002
:10182000809386009093870020E530E040E050E010
:1018300015D224E630E040E050E03CD22093640032
:1018400030936500409366005093670025E530E0D3
:1018500040E050E0C801B70101D224E630E040E0AA
:1018600050E028D2209360003093610040936200E2
:101870005093630084E096DB81E080930901ECCE15
:101880008091CB009091CC00A091CD00B091CE0082
:101890000196A11DB11D8093CB009093CC00A09325
:1018A000CD00B093CE000A97A105B10588F1109242
:1018B000CB001092CC001092CD001092CE0060911F
:1018C0000E0170910F0180911001909111012091F2
:1018D0000A0130910B0140910C0150910D01620FF2
:1018E000731F841F951F43DD872F90E0A0E0B0E0B9
:1018F00080930E0190930F01A0931001B0931101FA
:1019000081389105A105B1051CF481E08093CF00D9
:101910008091CF00882301F161E070E080E090E0E9
:101920009DD339D50BC061E084E0FCD36093910076
:101930007093920080939300909394008091910013
:1019400090919200A0919300B0919400885B9B408D
:10195000A040B04044F7DAC01ADC61E070E080E0FB
:1019600090E07CD31092C2001092C3001092C40089
:101970001092C5008091BE009091BF00A091C00060
:10198000B091C1000196A11DB11D8093BE0090933E
:10199000BF00A093C000B093C1008091C20090919D
:1019A000C300A091C400B091C5000196A11DB11D56
:1019B0008093C2009093C300A093C400B093C5006D
:1019C00061E084E0AFD37B018C0160939100709360
:1019D0009200809393009093940088EBE8168BE03C
:1019E000F80680E0080780E018078CF480918200F8
:1019F000813021F080918100823021F481E0809358
:101A0000810084C08091C600882309F47FC0809142
:101A10008100823029F080918200813009F05DC020
:101A20008091CB009091CC00A091CD00B091CE00E0
:101A30000A97A105B10508F0B0CF8091D0008823A6
:101A400009F0ABCF8091750090917600A09177005E
:101A5000B0917800880F991FAA1FBB1F2091C20068
:101A60003091C3004091C4005091C5008217930784
:101A7000A407B5070CF091CFDD24D394D092D00009
:101A800060910E0170910F018091100190911101F0
:101A90006E0D7F1D801F911F6ADC872F90E0A0E0F4
:101AA000B0E080930E0190930F01A0931001B093CA
:101AB00011010997A105B1050CF06FCF8AE090E004
:101AC000A0E0B0E08093CB009093CC00A093CD0039
:101AD000B093CE00D092CF0019C02091C2003091B7
:101AE000C3004091C4005091C50080917500909151
:101AF0007600A0917700B091780082179307A40731
:101B0000B5070CF04ACF81E08093C60048DAC6D210
:101B100064E670E080E090E0A1D289E288BB809129
:101B2000C600882349F46091C2007091C30080917F
:101B3000C4009091C500A8D862E08BE0F3D26D5745
:101B40007140804090402CF083E02CDA82E1809359
:101B500090001092C7001092C8001092C900109215
:101B6000CA0010920A0110920B0110920C011092FF
:101B70000D0180919000882309F46ECD64E670E039
:101B800080E090E06BD280919000803131F403D4FA
:101B900064EF71E080E090E061D28091900081314B
:101BA00061F4F9D364EF71E080E090E057D2F3D3B1
:101BB00064EF71E080E090E051D28091900082313A
:101BC00091F4E9D364EF71E080E090E047D2E3D391
:101BD00064EF71E080E090E041D2DDD364EF71E02A
:101BE00080E090E03BD2109290008091CF0088235B
:101BF00009F432CD1092D00061E070E080E090E016
:101C00002DD2C9D30BC061E084E08CD260939100E7
:101C10007093920080939300909394008091910030
:101C200090919200A0919300B0919400885B9B40AA
:101C3000A040B04044F710CD5527002480FF02C0DB
:101C4000060E571F660F771F6115710521F09695D7
:101C50008795009799F7952F802D0895FF27EE27F8
:101C6000BB27AA2760FF04C0A20FB31FE41FF51F04
:101C7000220F331F441F551F9695879577956795BB
:101C800089F70097760771F7CF01BD01089597FB9B
:101C9000092E07260AD077FD04D027D006D00020D1
:101CA0001AF4709561957F4F0895F6F79095819598
:101CB0009F4F089597FB092E05260ED057FD04D09F
:101CC00028D00AD0001C38F45095409530952195C5
:101CD0003F4F4F4F5F4F0895F6F790958095709561
:101CE00061957F4F8F4F9F4F0895AA1BBB1B51E1FA
:101CF00007C0AA1FBB1FA617B70710F0A61BB70B7C
:101D0000881F991F5A95A9F780959095BC01CD0120
:101D10000895A1E21A2EAA1BBB1BFD010DC0AA1F2C
:101D2000BB1FEE1FFF1FA217B307E407F50720F044
:101D3000A21BB30BE40BF50B661F771F881F991FBF
:101D40001A9469F760957095809590959B01AC0108
:081D5000BD01CF010895FFCF92
:101D58007C1500007017000050000000FEF4010020
:101D68000046000000CD00000064000000010000F3
:041D78000002020063
:00000001FF
